:100000000C943F020C9492020C9492020C94920273
:100010000C9492020C9492020C9492020C94920210
:100020000C9492020C9492020C945A200C9492021A
:100030000C949B2D0C9492020C9492020C949202BC
:100040000C9492020C9492020C9492020C949202E0
:100050000C9492020C94EC0A0C9492020C9492026E
:100060000C9492020C9492020C9492020C949202C0
:100070000C9492020C9492020C9492020C949202B0
:100080000C9492020C9492020C9492020C949202A0
:100090000C9492020C9492020C9492020C94920290
:1000A0000C9492020C9492020C949202A81ECF1E01
:1000B000C71FCF1EC71F1B1F3E1FC71F951FA41F93
:1000C000EA23EA23222422249D24D124C826C826F8
:1000D000E824C826792479248226C8269726B526BE
:1000E000808080800405060708090A0B0C0D0E0F9E
:1000F000101112131415161718191A1B1C1D1E1F88
:10010000202122232425262728292A2B2C2D2E2F77
:10011000303132333435363738393A3B3C3D3E3F67
:10012000404142434445464748494A4B4C4D4E4F57
:10013000505152535455565758595A5B5C5D5E5F47
:10014000606162636465736768696A6B6C6D6E6F2A
:100150007071727380808080808080808080800356
:100160000201808080668075007476778080808050
:100170007677808080808080808080808080808092
:10018000808080808080808080808080808080806F
:10019000808080808080808080808080808080805F
:1001A000808080808080808080808080808080804F
:1001B000808080808080808080808080808080803F
:1001C00078797A7B7C7D7E7F808080808080808053
:1001D000808080808080808080808080808080801F
:1001E00073706565643A2025730A007573625F73E6
:1001F000746174653A20253032580A00686F737450
:100200002E5461736B3A2025640A00526F6C6C6F38
:10021000766572206572726F723A2069676E6F72CE
:1002200065640D0A000D0A00202530325800696E01
:100230007075742025643A000A4B6579626F6172AB
:10024000642073746172742E0A000A55534220634D
:100250006F6E666967757265642E0A000A0A544DEE
:100260004B3A30323636346665372F4C5546410AA4
:100270000A003C03550053004200200074006F0048
:10028000200055005300420020006B0065007900FB
:1002900062006F00610072006400200063006F0064
:1002A0006E00760065007200740065007200000048
:1002B0000E0374002E006D002E006B002E00000057
:1002C0000403090409027400040100A032090400B7
:1002D0000001030101000921110100012240000772
:1002E00005810308000A0904010001030102000955
:1002F0002111010001224D000705820308000A09AF
:10030000040200010300000009211101000122364E
:10031000000705830308000A090403000203000024
:100320000009211101000122220007058403200099
:10033000010705040320000112011001000000085C
:10034000EDFE5B001408010200010631FF0974A1F3
:10035000010975150026FF009520750881020976B0
:10036000150026FF00952075089102C0050109803F
:10037000A10185021601002637001A81002AB70064
:10038000751095018100C0050C0901A101850316B6
:100390000100269C021A01002A9C02751095018119
:1003A00000C005010902A1010901A1000509190107
:1003B0002905150025019505750181029501750333
:1003C00081010501093009311581257F95027508E4
:1003D000810609381581257F950175088106050C70
:1003E0000A38021581257F950175088106C0C00570
:1003F000010906A101050719E029E7150025019566
:100400000875018102950175088101050819012906
:10041000059505750191029501750391010507196F
:100420000029FF150026FF00950675088100C029E8
:100430000A002575002F002575005D280025640041
:100440002000256400200025640020002564007C35
:100450000025303258006D6F7573656B6579205BD0
:1004600062746E7C782079207620685D28726570D1
:100470002F61636C293A205B00009C09570A112404
:100480001FBECFEFDAE0DEBFCDBF04B603FE28C04B
:100490008091D6059091D705A091D805B091D90546
:1004A0008730904BA740B04BD9F41092D6051092EC
:1004B000D7051092D8051092D90514BE0FB6F8943E
:1004C000A895809160008861809360001092600020
:1004D0000FBE1092010810920008E0E0F8E30995C1
:1004E00011E0A0E0B1E0E6EBF4E602C005900D9269
:1004F000AE39B107D9F725E0AEE9B1E001C01D92F0
:10050000A63DB207E1F712E0CFE3D2E004C02197A5
:10051000FE010E943F32CD33D107C9F70E94BD1BB7
:100520000C9459320C940000FF93EF93E0919E01DC
:10053000F0919F01309709F00995EF91FF9108958F
:10054000FC018591803011F0EFDFFBCF0895FF278C
:10055000E0E230E247FF0CC0419597FF09C0EDE2B1
:100560006095709580959095611D711D811D911DFF
:1005700027FF02C0219530E350E2AA27660F771FBC
:10058000881F991FAA1FA41710F0A41B63955A95E2
:10059000A9F7AA3008F0A95FA05DAF93F3956115A4
:1005A00071058105910541F7ED3211F4EF93F39553
:1005B000F21718F43F93F395FBCF8F91B5DFFA95BF
:1005C000E1F70895E991F9918591803021F0853224
:1005D00019F0AADFF9CF089520E0E894559155323B
:1005E000C1F3503311F4689455915A3348F4505381
:1005F00090F3220F022E220F220F200D250FF4CF91
:100600000EF4219589919991533619F3533729F1B5
:10061000533559F1BC0188279927E8945C3621F4B9
:100620008991999168945591543639F446EF7EF04A
:1006300077FF0DC08FEF9FEF0AC055374AE039F0C2
:10064000583540E121F0523642E009F00895FF9319
:10065000EF937DDFEF91FF91B7CFFF93EF93FC0115
:1006600081918030B9F360DFFBCFFF93EF9368DFB8
:10067000F1CFDF93CF93CDB7DEB72596A3DFCF9130
:10068000DF91089580E00895089580E0089581E065
:100690000895CF93DF93CDB7DEB728970FB6F894C0
:1006A000DEBF0FBECDBFE22F29833A834B835C832D
:1006B0006D837E838F8398878091DC02E82BE093A3
:1006C000DC02FE013396AE01475F5F4F219124307B
:1006D00088F0AEEDB2E080E090E03D91311106C0CF
:1006E000DC01A452BD4F12962C9304C001968630B3
:1006F000910599F7E417F50749F728960FB6F8948E
:10070000DEBF0FBECDBFDF91CF910895860F911D43
:10071000860F911DFC015687458781E00895FC01F5
:1007200087890895CF93DF93EC018C819D81DC0153
:10073000ED91FC910480F581E02D6E8109951F8675
:10074000188A81E08A8B1E821B8A1C8A1D8A1E8A57
:100750001F8A80E0DF91CF910895FC018681089582
:1007600081E0633009F080E0089581E0613009F0B4
:1007700080E00895860F911D860F911DFC018585EF
:1007800096850895EF92FF92CF93DF93DC01E70106
:1007900052968C915297823049F11F966C931F9715
:1007A00050964C9350979B8193709330F9F49A81B3
:1007B00097FF1CC09E8158962C915897291718F4C2
:1007C00058969C935897E82FF0E09F01220F331F13
:1007D000E20FF31FEA0FFB1F9A819F7097839C81A2
:1007E000908794E091878F5F52968C93DF91CF91A1
:1007F000FF90EF900895EF92FF920F9302970E945F
:10080000C2030F91FF90EF9008950895CF92DF9269
:10081000EF92FF920F931F93CF93DF93CDB7DEB785
:1008200062970FB6F894DEBF0FBECDBFDC015796BE
:100830002C91222381F06C010E946C0AF60103893D
:10084000148925893689DC01CB01801B910BA20B11
:10085000B30BB7FF02C0F12C3AC0838590E09A8BAE
:10086000898BE12C8E010F5F1F4F9E012F5E3F4F42
:1008700042856681848195810E94FD12F82E811146
:1008800018C029893A892330310598F0D6011D9680
:100890008D919C911E97009761F0DC01ED91FC9188
:1008A0000190F081E02D8E010F5F1F4F40E0B601F7
:1008B00009950E946C0AF601208DDC01CB01820FA4
:1008C000911DA11DB11D838B948BA58BB68B8F2D94
:1008D00062960FB6F894DEBF0FBECDBFDF91CF9109
:1008E0001F910F91FF90EF90DF90CF9008952F927E
:1008F0003F924F925F926F927F928F929F92AF92B0
:10090000BF92CF92DF92EF92FF920F931F93CF93FC
:10091000DF93CDB7DEB7EB970FB6F894DEBF0FBE0F
:10092000CDBFDC0116965C90511019C1422E242EC9
:10093000362E7C01FC01A480B580108ED501ED918E
:10094000FC910190F081E02D60E0C50109956C01FA
:10095000009719F446ED542E0FC1FC018080918060
:100960008114910409F4FEC03701F7E06F0E711C89
:10097000DC0111967C926E9214964C928E01065D6B
:100980001F4F28E030E040E060E0F701848195816E
:100990000E94BF10182F8111EBC01AA5D6018D92AD
:1009A0009C92D501ED91FC910280F381E02D222DE6
:1009B00040E0632DC5010995F7018683882309F47A
:1009C000D4C099A99087282F40E060E08481958168
:1009D0000E946A11982ED501ED91FC91D6011496D2
:1009E0001C92882361F00480F581E02DD7011696D2
:1009F0006C91C5010995F7011682592CBDC0019073
:100A0000F081E02DD70116966C91C50109950097EC
:100A100009F4A0CF212F133108F022E1FC01448218
:100A200021110FC03BAC412C36E2832E31E0932ED6
:100A30005701F2E0AF0EB11C6E0181E1C80ED11C6E
:100A400038C030E08E01065D1F4F40E0D70116969A
:100A50006C91169714968D919C9115970E94BF10DA
:100A6000182F811172C0DECF9A828982BC82AB823C
:100A70001D821A861B861E86188A1F8619A21AA234
:100A80001BA219A6DF82CE82D986C886DD86CC86D7
:100A90008E010F5F1F4F242D40E0F7016681848196
:100AA00095810E940D11D70152968C91823019F0D8
:100AB00043944310D9CFF7018289823009F044C0B2
:100AC000930142E06681848195810E943D0C68EE2D
:100AD00073E080E090E00E946E0AD7011F962C918F
:100AE0001F9740E016966C91169714968D919C91E5
:100AF00015970E94D812182F811127C068EE73E055
:100B000080E090E00E946E0AF701418D60E0C7012D
:100B10000E94E114182F811118C020E040E060E02D
:100B2000C7010E94B7148CE291E09A838983AE01D9
:100B30004F5F5F4F60E070E0C7010E94471481E0A3
:100B4000D70157968C9318C011EDD701ED91FC9108
:100B50000480F581E02DC7010995512E0DC029EDC6
:100B6000522E0AC097ED592E07C084ED582E04C0AE
:100B7000F60191828082E9CF852DEB960FB6F8942D
:100B8000DEBF0FBECDBFDF91CF911F910F91FF90C0
:100B9000EF90DF90CF90BF90AF909F908F907F901D
:100BA0006F905F904F903F902F9008953F924F929B
:100BB0005F926F927F928F929F92AF92BF92CF92ED
:100BC000DF92EF92FF920F931F93CF93DF9300D0AA
:100BD00000D0CDB7DEB76C017C836B835A83498329
:100BE0004C0180E1880E911C5601A7E0AA0EB11CB1
:100BF00011E084E0482E3601B2E16B0E711C93E0E7
:100C0000392E22E0522E8B819C81892B09F4FBC066
:100C1000F60180A1823059F128F4882341F0813017
:100C200071F0F1CF833039F18430C1F1ECCF5482CF
:100C300085819681908787835286518610A3AE0165
:100C40004D5F5F4FBE016F5F7F4FC5010E94D5189A
:100C5000882309F4D8C0D6011596ED91FC9116971A
:100C6000808191968C939197818192968C93F601D5
:100C70007682658230A2D60192968C9192978430CA
:100C800011F493961C92F60181A1825084832581F0
:100C90003681308727838287818740A2D60192964A
:100CA0008C918430B1F0853009F442C0823009F073
:100CB0006EC0AE014D5F5F4FBE016F5F7F4FC501DC
:100CC0000E94D518882309F49EC0F601858984A363
:100CD00092C0AE014D5F5F4FBE016F5F7F4FC50198
:100CE0000E94D518882309F48EC0D60155968C91A0
:100CF0005597833009F07FC056968C915697813076
:100D000009F079C098969C91989757968C91992361
:100D100021F0882309F46FC003C0813009F06BC053
:100D2000F60113A3928996A3938997A385A363C021
:100D3000AE014D5F5F4FBE016F5F7F4FC5010E94E7
:100D4000D518882309F45FC0D60193968C919397A8
:100D5000882309F450C012968D919C9113970097A7
:100D600009F449C0DC01ED91FC910190F081E02D86
:100D70007401D60195960C91959797962C9197971B
:100D800096964C91969794966C91099534C0F6017D
:100D90008585882319F0813039F028C081A190E041
:100DA00002979787868715872B813C8189819A8155
:100DB000782F692FF601468557854115510581F039
:100DC00001962115310529F41C821B8279836A83DF
:100DD0000DC0415051095787468721503109E8CF4E
:100DE0003C832B839A838983F6011586F6018685D9
:100DF0009785892B41F4D60116969C928E92159771
:100E000090961C9200CF0F900F900F900F90DF9153
:100E1000CF911F910F91FF90EF90DF90CF90BF90F7
:100E2000AF909F908F907F906F905F904F903F908A
:100E30000895CF93DF936091FA017091FB01E091E7
:100E4000A701F091A8014091EE015091EF0120918E
:100E5000E2013091E3018091D6019091D7016E17A4
:100E60007F07B1F4E091A501F091A6014E175F074D
:100E700079F4E091A301F091A4012E173F0741F40A
:100E8000E091A101F091A2018E179F0709F463C0C0
:100E90007093A8016093A7015093A6014093A50108
:100EA0003093A4012093A3019093A2018093A10108
:100EB000ECEDF2E088E0DF011D928A95E9F72091E0
:100EC000F2013091F3014091F4015091F5016091EC
:100ED000F6017091F7018091F8019091F9010E945B
:100EE00049032091E6013091E7014091E8015091DA
:100EF000E9016091EA017091EB018091EC01909120
:100F0000ED010E9449032091DA013091DB0140910B
:100F1000DC015091DD016091DE017091DF01809173
:100F2000E0019091E1010E9449032091CE013091AE
:100F3000CF014091D0015091D1016091D2017091C7
:100F4000D3018091D4019091D5010E94490381E0A1
:100F50008093DB0202C01092DB020E94C50AEC0102
:100F600084E692E00E943613CE010E94DD0A8536A7
:100F7000910560F09F938F938CEF91E09F938F93F7
:100F80000E9439030F900F900F900F9084E692E02B
:100F90000E941D0C9091A001891779F184E692E0DE
:100FA0000E941D0C8093A0011F928F938BEE91E005
:100FB0009F938F930E9439030F900F900F900F9083
:100FC0008091A0018039C9F48091A901823019F083
:100FD0008EE191E002C089E191E09F938F9380EED2
:100FE00091E09F938F930E9439030E9448210E94B1
:100FF00041220F900F900F900F9081E0DF91CF91E1
:101000000895482F80E1489F90011124205E310906
:101010002830310538F49091DC02992319F0892F9A
:1010200090E002C080E090E0EEEDF2E061E070E080
:101030002191243070F0322F32953F70431309C054
:101040002F70DB0102C0AA0FBB1F2A95E2F78A2B83
:101050009B2BB2E0E43EFB0759F708950895CF9229
:10106000DF92EF92FF920F93CF93DF931F92CDB752
:10107000DEB7898380916102882371F0CE010196E9
:101080006C01EE24E394F12C00E022E040E060E00B
:101090008AE492E00E948A1480914702882371F0CA
:1010A000CE0101966C01EE24E394F12C00E022E0E5
:1010B00040E060E080E392E00E948A1480912D027B
:1010C000882371F0CE0101966C01EE24E394F12C9B
:1010D00000E022E040E060E086E192E00E948A14B5
:1010E00080911302882371F0CE0101966C01EE24E9
:1010F000E394F12C00E022E040E060E08CEF91E02E
:101100000E948A140F90DF91CF910F91FF90EF9082
:10111000DF90CF9008950E94592D8091CB058823B0
:1011200031F00E94822D882321F00C94D61C0C945F
:1011300019070895FC017583648382E391E091832C
:10114000808380E591E093838283138A148A158AD1
:10115000168A178A418F178288E080878CE38187FF
:101160001286138684E0848781E0828B118A178639
:101170001686158661157105B1F0DB01AA5ABF4FBD
:1011800080E090E02D913D91232B49F48B96880FC0
:10119000991FDB01A80FB91FED93FC9308950196E9
:1011A0008031910579F708952E9A08952E988EBD75
:1011B0000DB407FEFDCF1EBC0DB407FEFDCF0E948F
:1011C000D4088EB508952E9882608EBD0DB407FEAA
:1011D000FDCF6EBD0DB407FEFDCF0C94D40888EF93
:1011E0000E94D608807C803411F118F4882371F1B4
:1011F0000895803819F0803C39F1089588ED0E94F7
:10120000D6089091A90181FD08C0923029F161ECC6
:1012100088ED0E94E30882E007C09330E9F063ECB8
:1012200088ED0E94E30883E08093A901089588ED8A
:101230000E94D6089091A90181FD03C0933079F7EF
:101240000895923021F7089581E0EECF61ED88EDA9
:101250000E94E3081092A90108950F931F93CF9362
:10126000DF938C01269A0E94D408219A229A23980F
:10127000209A80E58CBD81E08DBD259868E188E8E5
:101280000E94E30860E288E70E94E30860E088E7E4
:101290000E94E308C0E0D0E088E60E94D6082196CC
:1012A00080FD06C0CF3F8FEFD807B1F78FEF1DC08D
:1012B00061EC88ED0E94E30860E280ED0E94E308A3
:1012C00064E088EE0E94E30888EE0E94D60882FF60
:1012D000FBCFC8010E94EF0860E288EC0E94E3089F
:1012E00061E080E80E94E30880E0DF91CF911F91E8
:1012F0000F9108958091BE0581608093BE0584E6BC
:1013000092E00E942D0980EF91E090935802809323
:10131000570284EE91E090933E0280933D0288ED67
:1013200091E090932402809323028CEC91E09093BF
:101330000A0280930902089584E692E00E94ED0B70
:1013400040E064E672E08AE492E00E949A0840E09D
:1013500064E672E080E392E00E949A0840E064E66E
:1013600072E086E192E00E949A0840E064E672E052
:101370008CEF91E00E949A0886E591E09093F1014C
:101380008093F0019093E5018093E4019093D9015B
:101390008093D8019093CD018093CC0164E672E0F4
:1013A0008BEB91E00E94651764E672E08AEA91E0B7
:1013B0000C946517AF92BF92CF92DF92EF92FF929B
:1013C0000F931F93CF93DF937C01CB01D22EDB01D0
:1013D000ED91FC910084F185E02D09951F928F938A
:1013E0008EE292E09F938F930E943903E8015801A7
:1013F000AD0CB11C0F900F900F900F9088E2C82E8B
:1014000082E0D82ECA15DB0561F089911F928F9377
:10141000DF92CF920E9439030F900F900F900F90A0
:10142000F1CF85E292E09F938F930E9439030F9052
:101430000F90F8018281813049F48BE092E09F9314
:101440008F930E9439030F900F900FC0D70112960F
:1014500088E0F80101900D928A95E1F70E946C0AEC
:10146000D7011B967C936E931A97DF91CF911F91B2
:101470000F91FF90EF90DF90CF90BF90AF900895C5
:1014800080E090E008958FEF9FEF089581E090E075
:1014900008950895862F0E94DE1981E090E0089556
:1014A000FB0180810E94DE1981E090E00895E4EE66
:1014B000F2E01382128288EE93E0A0E0B0E0848331
:1014C0009583A683B7838CE591E0918380838FEF2A
:1014D0009FEF9587848708950C94D10A8F929F92ED
:1014E000AF92BF92CF92DF92EF92FF920E940731AC
:1014F0004B015C0120E030E04AE755E40E94BE3138
:101500006B017C0120E030E040E85FE30E94CC30DA
:1015100087FD24C020E03FEF4FE757E4C701B60145
:101520000E94B9311816ACF420E030E040E251E4FA
:10153000C501B4010E94BE310E94D83020E931E0DB
:101540006115710581F0C9010197F1F761507109C9
:10155000F7CFC701B6010E94D83002C061E070E049
:10156000CB010197F1F7FF90EF90DF90CF90BF9004
:10157000AF909F908F90089582E084BD93E095BDD9
:101580009AEF97BD80936E0008952FB7F8948091DD
:10159000340390913503A0913603B09137032FBFE8
:1015A00008952FB7F89460913403709135038091BA
:1015B0003603909137032FBF08959C014FB7F894DD
:1015C0008091340390913503A0913603B091370395
:1015D0004FBF821B930B089578941F920F920FB602
:1015E0000F9211248F939F93AF93BF9380913403F5
:1015F00090913503A0913603B09137030196A11D58
:10160000B11D8093340390933503A0933603B093B8
:101610003703BF91AF919F918F910F900FBE0F90A5
:101620001F901895CF93DF93FC01862F8078A9F443
:10163000283008F04DC0442321F09581973009F4FB
:1016400047C0EF01A1E0B0E09D85992341F01196DC
:101650002596A031B105C1F73BC080E039C06111CA
:101660001CC085E08A9FE0018B9FD00D1124CE0F16
:10167000DF1F442331F081E4888785818F5F858374
:1016800002C081E0888725E02A9FC0012B9F900D32
:101690001124E80FF91F80851BC06770660F660F65
:1016A000660F442341F0606485818F5F8583877076
:1016B000687F682B03C02770687B622B25E02A9F18
:1016C000C0012B9F900D1124E80FF91F6087862F12
:1016D000DF91CF910895611102C006960895FC0133
:1016E00021E03585631739F02F5F35962031C9F732
:1016F00080E090E00895069635E0239F800D911DCF
:1017000011240895DF92EF92FF920F931F93CF93CE
:10171000DF93EC01E62EF12C85E0689FB0011124E7
:10172000FE01E60FF71F8085182F177086FF17C080
:1017300001E085E0D82EFE01D09EE00DF11D1124C0
:10174000808586958695869587701817F9F00F5FC6
:10175000003189F78D81811302C011501D8385E00E
:101760008E9DF0018F9DF00D1124EC0FFD1F108652
:1017700081E0818712862296D783C683DF91CF913D
:101780001F910F91FF90EF90DF900895602FCE0191
:101790000E94820BD0CFFC01613499F49C01255B3F
:1017A0003F4F61E0AC014E5F5F4F1586668717863D
:1017B000548743873596E217F307B9F7FC01158282
:1017C000089521E03585631729F02F5F3596203184
:1017D000C9F70895622F0C94820BFC018EE691E00C
:1017E000918380831582108681E081871286CF01E4
:1017F000029697838683128228E023832CE3248336
:10180000DF019F01255B3F4F41E01D961C921D9714
:101810001E964C931E971F961C921F971C969C9386
:101820008E931B971596A217B30779F7EA58FF4FC7
:10183000108281E180933C03089580913C030895D8
:10184000CF93C42F0E946B0B009789F0DC01ED91C0
:10185000FC911197309759F013969C9180E089176D
:1018600031F020812C1731F033968F5FF8CF80E074
:1018700090E001C0CF01CF9108950F931F93CF93B4
:10188000DF932115310571F0E901042F162F0E9415
:101890006B0BFC01892B41F01283D183C08303833E
:1018A00080E003C088ED01C086EDDF91CF911F91EC
:1018B0000F910895CF92DF92FF920F931F93CF93D2
:1018C000DF93662381F1F62E8C016C0186E5C80E4C
:1018D000D11CC0E0D0E0D6018D919D916D010097A3
:1018E000F1F0DC01ED91FC910084F185E02D09958A
:1018F000F81215C0AB96CC0FDD1FC00FD11F888129
:101900009981DC01ED91FC910480F581E02DDF915E
:10191000CF911F910F91FF90DF90CF900994219666
:10192000C031D105C1F680E0DF91CF911F910F91B9
:10193000FF90DF90CF9008952E980895CF93C82FF1
:101940000E949C0CCEBD0DB407FEFDCF1EBC0DB495
:1019500007FEFDCF0E94D4088EB5CF910895CF9396
:10196000DF93C82FD62F0E949C0CC260CEBD0DB451
:1019700007FEFDCFDEBD0DB407FEFDCFDF91CF9199
:101980000C94D4088F929F92AF92BF92CF92DF9225
:10199000EF92FF920F931F93CF93DF93EC01D62E1C
:1019A000C42E59010E946B0B7C01009709F445C0BD
:1019B000FC0180819181892B09F441C04C2D6D2D52
:1019C000CE010E94200CF501918380830097C9F11C
:1019D000FC0182818695869590E08031910514F016
:1019E0008FE090E041E050E060E070E04A015B0190
:1019F00004C0880C991CAA1CBB1C8A95D2F7D5017F
:101A0000C4010197F801918380836D2D80EE0E94BF
:101A1000AF0C88ED0E949E0CF7019481992331F060
:101A2000CA58DF4F68816260682B02C0682F697FE7
:101A300088ED0E94AF0C80E005C086ED03C087ED05
:101A400001C08BEDDF91CF911F910F91FF90EF902F
:101A5000DF90CF90BF90AF909F908F9008958F921E
:101A60009F92AF92BF92CF92DF92EF92FF920F932D
:101A70001F93CF93DF93862E942E59010E946C0AF8
:101A80006B017C0128E8C20E23E1D21EE11CF11C8F
:101A900000E010E0D0E0C0E098280E946C0ADC0171
:101AA000CB018C199D09AE09BF09B7FF2DC0692D67
:101AB00080EF0E94AF0C0E946C0ADC01CB018C19F4
:101AC0009D09AE09BF09B7FF09C088EC0E949E0CB2
:101AD00087FFF1CF60E888EC0E94AF0C88EF0E948E
:101AE0009E0CC82FCF70C43019F0CE3051F00CC00E
:101AF0000F5F1F4FA114B10481F20A151B0569F68F
:101B000003C0DF5FD33049F68C2FDF91CF911F9157
:101B10000F91FF90EF90DF90CF90BF90AF909F908C
:101B20008F9008959F92AF92BF92CF92DF92EF92E3
:101B3000FF920F931F93CF93DF937C01D42F122F2B
:101B4000902E00E06C01C60ED11CC60ED11C86E59D
:101B5000C80ED11CA42EB12CABE2AA0EB11CAA0C4B
:101B6000BB1CAE0CBF1CF60180819181DC01ED91A4
:101B7000FC910280F381E02D292D412F6D2F0995D5
:101B8000803EC9F4D1110BC061E088EE0E94AF0C19
:101B900066E670E080E090E00E946E0A14C0F501F5
:101BA00080819181DC01ED91FC910284F385E02D2F
:101BB000612F099508C08D3021F4033008F03FC033
:101BC00014C081113FC0F60180819181DC01ED914B
:101BD000FC910190F081E02D292D412F6D2F099569
:101BE000C82F8D3051F4033050F464E670E080E08B
:101BF00090E00E946E0A0F5FB6CF882311F1D111D9
:101C00000BC061E088EE0E94AF0C66E670E080E0F9
:101C100090E00E946E0A11C0ED2FF0E0BB96EE0F2F
:101C2000FF1FEE0DFF1D80819181DC01ED91FC9184
:101C30000284F385E02D612F09958C2F03C08DE080
:101C400001C080E0DF91CF911F910F91FF90EF9045
:101C5000DF90CF90BF90AF909F9008950F931F9308
:101C6000CF93DF93182F062FEA010E949C0C12607D
:101C70001EBDFE01802F882339F00DB407FEFDCF75
:101C800091919EBD8150F7CFC00FD11D0DB407FEBD
:101C9000FDCF0E94D408CE01DF91CF911F910F910B
:101CA00008952F923F924F925F926F927F928F9200
:101CB0009F92AF92BF92CF92DF92EF92FF920F93DB
:101CC0001F93CF93DF9300D000D01F92CDB7DEB724
:101CD0007B014A016901FB01F181F9838F2F81505A
:101CE000803408F075C00E946C0A2B013C0128E882
:101CF000420E23E1521E611C711CF701828180FD9E
:101D000002C060E401C060E888EE0E94AF0C312C94
:101D10009981892F90E09A838983C114D10409F4B1
:101D20004AC0E981FA81FD83EC83CE16DF0610F408
:101D3000DD82CC82FC81FB83A8016F2F80E10E94B1
:101D40002E0E6C8188E30E94AF0CF7016081606207
:101D500080EF0E94AF0C88EC0E949E0C87FFFBCFA7
:101D600060E888EC0E94AF0C88EF0E949E0C8F7098
:101D7000382EA12CB12C212C332009F451C00E9403
:101D80006C0ADC01CB0184199509A609B709B7FFD4
:101D900047C0F6E03F1611F12EE03216D9F084E08C
:101DA000381209C0FFEFAF1ABF0A81149104B1F0D5
:101DB000A814B90499F488EF0E949E0C85FB88272B
:101DC00080F9F701928180FB90F99283832D2FC0D7
:101DD0008AED2DC0239423E0221669F360E088E3A6
:101DE0000E94AF0CF801608180E10E94AF0C6B8112
:101DF00088E30E94AF0CF7016081606280EF0E946F
:101E0000AF0C88EC0E949E0C87FFFBCF60E888EC4B
:101E10000E94AF0C88EF0E949E0C8F70382EACCFC2
:101E2000EC81FD81CE1ADF0A0E0F1F1F76CF0F90B7
:101E30000F900F900F900F90DF91CF911F910F9106
:101E4000FF90EF90DF90CF90BF90AF909F908F90DA
:101E50007F906F905F904F903F902F9008952F92BA
:101E60003F924F925F926F927F928F929F92AF922A
:101E7000BF92CF92DF92EF92FF920F931F93CF9377
:101E8000DF93CDB7DEB72A970FB6F894DEBF0FBE4B
:101E9000CDBF9D838C836B015F834E835901EA82A2
:101EA000F90180809180FB01F181FB83F9011182AE
:101EB0001082FB01828181FD02C060E101C060E20D
:101EC00088EE0E94AF0C8886FA814F2E512C612C2F
:101ED000712C2E813F81F601408160E08C819D81D3
:101EE0000E942F0D89838630A1F3811163C088EC95
:101EF0000E949E0C82FF5CC080E30E949E0C382EE4
:101F000090E08816990608F43884F5018081918163
:101F10009401281B390B3A87298737FF02C01A869C
:101F20001986E32CF12C89859A85E816F90614F4B4
:101F3000FA86E98629840E949C0C98E09EBD0DB427
:101F400007FEFDCFF801222041F01EBC2A940DB4FB
:101F500007FEFDCF8EB58193F6CFE985FA850E0F8A
:101F60001F1F0E94D40864E088EC0E94AF0CF501AA
:101F700080819181E80EF91EF182E082FB813F169B
:101F800018F0E814F90458F088EF0E949E0C82952E
:101F90008170F601928180FB91F992830BC0FA81E6
:101FA000FF2309F496CFC301B2010E946E0A91CFBC
:101FB00020EF298389812A960FB6F894DEBF0FBEE1
:101FC000CDBFDF91CF911F910F91FF90EF90DF90E8
:101FD000CF90BF90AF909F908F907F906F905F90C9
:101FE0004F903F902F9008952F923F924F925F9283
:101FF0006F927F928F929F92AF92BF92CF92DF9219
:10200000EF92FF920F931F93CF93DF93CDB7DEB77D
:1020100061970FB6F894DEBF0FBECDBF3C01F42E22
:10202000322E202EC98A4EA05FA0C8A4D9A4188A37
:102030001F861E861D868E01035F1F4F9E01215F36
:102040003F4F0E94C20C811181C039822A82EB82EB
:1020500089898C83BE82AD8298868F82AE014F5F64
:102060005F4F68E080E20E942E0E2D853E854F2D49
:1020700060E1C3010E942F0D182F811163C0932DC1
:102080009078392EC114D10409F44DC0EF85F88938
:1020900082819923C9F1826082835401A114B10421
:1020A00009F446C05C864B864D855E856F857889D0
:1020B000E12C86019E01255F3F4FC3010E942F0F37
:1020C000182F863059F381113DC0AAA5BBA51097E2
:1020D00099F0ED91FC9111970190F081E02DC401F0
:1020E0008A199B099A8789876B857C859E01275F62
:1020F0003F4FA601CD0109958B859C85A81AB90A89
:102100008415950558F60FC0816082834D855E85E4
:1021100086019201BF01C3010E94510E811116C0B8
:102120002D853E8511C02D853E85311005C00CC022
:10213000111108C02D853E8560EA4F2DC3010E9414
:102140002F0D04C0812F02C060E8F7CF61960FB653
:10215000F894DEBF0FBECDBFDF91CF911F910F91DD
:10216000FF90EF90DF90CF90BF90AF909F908F90B7
:102170007F906F905F904F903F902F9008958F9237
:102180009F92AF92BF92CF92EF920F931F931F92A5
:102190001F921F930F933F932F934901A12CB12CB2
:1021A000CC24C394E12C06E020E80E94F40F0F90A9
:1021B0000F900F900F900F900F901F910F91EF9035
:1021C000CF90BF90AF909F908F9008958F929F92E5
:1021D000AF92BF92CF92EF92FF920F931F921F92F6
:1021E000FF92EF923F932F934901A12CB12C22E053
:1021F000C22EE02E06E020E80E94F40F0F900F9010
:102200000F900F900F900F900F91FF90EF90CF9045
:10221000BF90AF909F908F9008954F925F926F9272
:102220007F928F929F92AF92BF92CF92DF92EF9266
:10223000FF920F931F93CF93DF93CDB7DEB7C054B8
:10224000D1090FB6F894DEBF0FBECDBF3C01D62E2C
:10225000542E422EC02ECE0101965C017C01022F2D
:1022600029E030E0C3010E94E61081111BC08B8081
:102270009C801F93CF92BF92AF921F9280E48F9366
:10228000A12CB12C82E0C82EE42C06E020E8452DDC
:102290006D2DC3010E94F40F0F900F900F900F90BF
:1022A0000F900F90C05CDF4F0FB6F894DEBF0FBEEB
:1022B000CDBFDF91CF911F910F91FF90EF90DF90F5
:1022C000CF90BF90AF909F908F907F906F905F90D6
:1022D0004F9008958F929F92AF92BF92CF92EF92BC
:1022E0000F93CF931F921F921F921F921F921F92C4
:1022F000812C912CA12CB12CC12CE22E05E020E0E8
:102300000E94F40FC82F6CE271E080E090E00E9420
:102310006E0A0F900F900F900F900F900F908C2FD0
:10232000CF910F91EF90CF90BF90AF909F908F90F3
:1023300008950F931F93CF93DF938A3F3FEF930747
:1023400011F486ED2DC0DC011696ED91FC911797E6
:10235000EF2B09F1122F242FEC011A8740E00E9485
:10236000120B082F8823C9F0682FCE010E946B0B37
:10237000009739F3FC011483202F40E060E0CE0188
:102380000E946A11182F882351F0602FCE010E94FD
:10239000CB0B812F05C087ED03C084ED01C080E029
:1023A000DF91CF911F910F9108952F923F924F92FD
:1023B0005F926F927F928F929F92AF92BF92CF92D5
:1023C000DF92EF92FF920F931F93CF93DF93CDB7DE
:1023D000DEB766970FB6F894DEBF0FBECDBF1B8A7F
:1023E00038E03C8B3CE33D8B8A3F3FEF930709F499
:1023F00064C0522E342E462E7C01DC011696CD9000
:10240000DC901797CE01439617969C938E93169760
:102410001A962C938E010F5F1F4F22E130E040E0AF
:1024200060E0C7010E94BF10F701D782C682811108
:10243000A6C089849A846B847C84FD81FE8B2E8067
:10244000670136E5C30ED11C560110E0D5018D9110
:102450009C910097F1F1DC01ED91FC910084F185F4
:10246000E02D0995811135C0F50180819181DC0154
:10247000ED91FC910088F189E02D622D099588236A
:1024800041F1F50180819181DC01ED91FC910484A1
:10249000F585E02DA301B4010995811110C0F50166
:1024A00080819181DC01ED91FC910684F785E02D1E
:1024B0006E890995811103C00CC086ED60C0052DA1
:1024C000232D442D612FC7010E94920D813D09F0FB
:1024D00056C01F5FB2E0AB0EB11C103109F0B6CF91
:1024E00010E0F601808191810097E1F1DC01ED912E
:1024F000FC910084F185E02D0995811133C0F6012E
:1025000080819181DC01ED91FC910088F189E02DC1
:10251000622D09958823D9F0F60180819181DC0133
:10252000ED91FC910484F585E02DA301B40109959A
:10253000811118C0F60180819181DC01ED91FC913F
:102540000684F785E02D6E89099581110BC0052D54
:10255000232D442D612FC7010E94920D982F977F44
:10256000913D69F41F5FE2E0CE0ED11C103109F0FD
:10257000B8CF252D432D642DC7010E949911669671
:102580000FB6F894DEBF0FBECDBFDF91CF911F9184
:102590000F91FF90EF90DF90CF90BF90AF909F9002
:1025A0008F907F906F905F904F903F902F90089505
:1025B0008F929F92AF92BF92CF92EF920F931F9202
:1025C0001F921F921F921F921F92812C912CA12C5F
:1025D000B12CC12CE22E09E020E00E94F40F0F90F4
:1025E0000F900F900F900F900F900F91EF90CF9052
:1025F000BF90AF909F908F9008958F929F92AF92CF
:10260000BF92CF92DF92EF920F931F93CF93DF93FE
:1026100000D000D0CDB7DEB76C01590148011C8253
:102620001B821A8219828E010F5F1F4F9E012D5F40
:102630003F4F0E94C20C811109C049815A816B81B0
:102640007C8184019501C6010E942F0F0F900F908D
:102650000F900F90DF91CF911F910F91EF90DF902E
:10266000CF90BF90AF909F908F900895AF92BF9200
:10267000CF92DF92EF92FF920F931F93CF938C0133
:102680001D990EC088EC0E949E0C85FF05C0C801F4
:102690000E94EF0860E201C060E088EC0E94AF0C8D
:1026A0008091A901813039F040F0823079F0833097
:1026B00079F5C1E00CC083E106C080913C03807FC6
:1026C000803131F181E180933C0322C0C0E08091F0
:1026D0003C03807F8031E9F40E946C0ADC01CB016D
:1026E00088539F4FAF4FBF4F809338039093390368
:1026F000A0933A03B0933B0380E280933C0380EDC8
:102700000E949E0C682F6F7D80ED0E94AF0C01C06F
:10271000C0E0780186E5E80EF11C6801A6E7CA0E64
:10272000D11C5701F501819191915F01009739F01A
:10273000DC01ED91FC910680F781E02D0995AC1448
:10274000BD0481F780913C03803409F447C050F404
:10275000803221F18033A1F1813109F08EC0F60180
:1027600010820AC0813509F464C0803809F476C04B
:10277000803509F082C045C0D7018D919D917D01C2
:10278000009739F0DC01ED91FC910480F581E02D9A
:102790000995EC14FD0481F782E16DC00E946C0A7A
:1027A000009138031091390320913A0330913B0393
:1027B000DC01CB01801B910BA20BB30BB7FD5DC0FD
:1027C00080ED0E949E0C682F606280ED0E94AF0C2D
:1027D00061E088EE0E94AF0C80E44DC088EE0E945C
:1027E0009E0C80FD4AC060E488EC0E94AF0C88ED2E
:1027F0000E949E0C682F686088ED0E94AF0C80E5F7
:102800003AC088EC0E949E0C86FF37C081E5809319
:102810003C030E946C0ADC01CB014496A11DB11D52
:102820008093380390933903A0933A03B0933B030A
:1028300024C00E946C0AC0903803D0903903E09005
:102840003A03F0903B03DC01CB018C199D09AE09E2
:10285000BF09B7FD12C080E880933C032C2F40E0F5
:1028600060E0C8010E94D511882321F0823D29F043
:1028700080EA01C080E980933C03CF911F910F91C2
:10288000FF90EF90DF90CF90BF90AF9008958F9220
:102890009F92AF92BF92CF92EF920F93CF93DF931D
:1028A000CDB7DEB7C054D1090FB6F894DEBF0FBE66
:1028B000CDBF5F934F939E012F5F3F4F3F932F9369
:1028C0001F9220E42F9320E8822E912C5B0132E2AC
:1028D000C32EE12C06E021E840E0FC016681848102
:1028E00095810E94F40F0F900F900F900F900F9012
:1028F0000F90C05CDF4F0FB6F894DEBF0FBECDBFA8
:10290000DF91CF910F91EF90CF90BF90AF909F90BC
:102910008F9008958F929F92AF92BF92CF92DF9245
:10292000EF92FF920F93A42EB12C1F921F92DF9271
:10293000CF92FF92EF924701C22EE02E09E021E2F2
:10294000462FFC016681848195810E94F40F0F90CF
:102950000F900F900F900F900F900F91FF90EF90AE
:10296000DF90CF90BF90AF909F908F9008958F92FF
:102970009F92AF92BF92CF92EF920F93A62EB12C5F
:102980001F921F921F921F921F921F92812C912CB7
:10299000C22EE42E0AE021E240E0FC01668184813F
:1029A00095810E94F40F0F900F900F900F900F9051
:1029B0000F900F91EF90CF90BF90AF909F908F901E
:1029C00008958F929F92AF92BF92CF92EF920F9302
:1029D000A62EB12C1F921F921F921F921F921F9220
:1029E000812C912CC12CE42E0BE021E240E0FC0173
:1029F0006681848195810E94F40F0F900F900F9053
:102A00000F900F900F900F91EF90CF90BF90AF90DD
:102A10009F908F900895FC018285089581E0693030
:102A200009F080E00895CF93DF93EC018A819B81C8
:102A3000DC01ED91FC910480F581E02D6A8509951A
:102A40008A85813439F4EA81FB81EA58FF4F80811D
:102A50008B7F80831A861B861C861D861E861F869A
:102A6000188A80E0DF91CF9108958F929F92AF9264
:102A7000BF92CF92EF920F93A42EB12CB22A1F9245
:102A80001F921F921F921F921F92812C912CC12C7A
:102A9000E62E01E023E240E0FC0162858281938121
:102AA0000E94F40F0F900F900F900F900F900F90C7
:102AB0000F91EF90CF90BF90AF909F908F9008951F
:102AC0008F929F92AF92BF92CF92EF920F93A62ECA
:102AD000B12C1F921F923F932F935F934F934A0104
:102AE000C12CE12C00E023EA40E0FC0162858281F8
:102AF00093810E94F40F0F900F900F900F900F9002
:102B00000F900F91EF90CF90BF90AF909F908F90CC
:102B100008958F929F92AF92BF92CF92EF920F93B0
:102B2000A42EB12CB22A1F921F921F921F921F92A5
:102B30001F92812C912CC12CE62E03E023E240E071
:102B4000FC016285828193810E94F40F0F900F90A7
:102B50000F900F900F900F900F91EF90CF90BF902C
:102B6000AF909F908F9008952F923F924F925F92D7
:102B70006F927F928F929F92AF92BF92CF92DF928D
:102B8000EF92FF920F931F93CF93DF93CDB7DEB7F2
:102B9000E8970FB6F894DEBF0FBECDBFDC011A96E2
:102BA0003C91311107C1122F242E362E3C01FC011D
:102BB000C280D380D601ED91FC910190F081E02D8F
:102BC00060E0C60109957C01009709F4F5C0FC019D
:102BD000A080B180A114B10409F4F0C04301F4E075
:102BE0008F0E911CDC0111969C928E9214961C9370
:102BF000FE0131962F018F0128E030E040E060E0D7
:102C0000D30112968D919C9113970E94BF10F701EA
:102C100014828111D9C08D81893009F0D1C0098118
:102C2000D601ED91FC910280F381E02D222D41E04F
:102C3000632DC6010995F3018287882309F4C2C078
:102C400098859583282F40E060E0828193810E94DF
:102C50006A11182F882389F0D701AD92BC92D60152
:102C6000ED91FC910480F581E02DD3011A966C91D1
:102C7000C6010995F3011286ABC0202F013208F07E
:102C800020E2D701AD92BC9221110BC0940142E029
:102C9000F3016285828193810E943D0C811197C06E
:102CA00010C030E0820140E0D3011A966C911A976F
:102CB00012968D919C9113970E94BF10811187C02D
:102CC000E5CF1F921F925F924F921F9288E08F93E1
:102CD00088E0882E912CA12CB12C99E2C92EE12CF0
:102CE00006E020EA40E0F3016285828193810E9440
:102CF000F40F182F0F900F900F900F900F900F90D0
:102D0000811166C08B81D3011B968C931B97720136
:102D100000E028E030E040E01A966C911A97129695
:102D20008D919C9113970E94E610811150C02B81C8
:102D30003C8140E0F3016285828193810E94E6102C
:102D4000811145C0298130E0CE0181967C0140E0AF
:102D5000D3011A966C911A9712968D919C911397A4
:102D60000E94E610811133C02E8140E0F30162859C
:102D7000828193810E94D812811129C001E0D30180
:102D80001B968C91801740F020E0402F68E0C30133
:102D90000E9489150F5FF3CFD3011296ED91FC913C
:102DA0001397EA58FF4F80818460808381E05096BA
:102DB0008C930EC019ED0CC016ED0AC017ED08C0BB
:102DC00011ED06C014ED04C0F701B182A082182FE6
:102DD000812FE8960FB6F894DEBF0FBECDBFDF910E
:102DE000CF911F910F91FF90EF90DF90CF90BF9008
:102DF000AF909F908F907F906F905F904F903F909B
:102E00002F900895CF92DF92FF920F931F93CF934D
:102E1000DF9300D000D0CDB7DEB78C01F62E19823B
:102E20001A821B821C8220E0462F61E10E94351528
:102E300020E04F2D60E1C8010E94351520E04F2DA4
:102E400064E0C8010E94891583E0C82ED12C9E0140
:102E50002F5F3F4F44E050E06F2DC8010E94601586
:102E60008823F1F020E04F2D64E1C8010E94351560
:102E700020E04F2D60E1C8010E94351564E170E04B
:102E800080E090E00E946E0A0F900F900F900F90DC
:102E9000DF91CF911F910F91FF90DF90CF90089518
:102EA00089819A81AB81BC819D7F83309140A04113
:102EB000B105C1F264E670E080E090E00E946E0A25
:102EC00081E0C81AD10819F6CDCFFC0188E791E05E
:102ED000918380837383628312861386148615869A
:102EE00016861786108A148288E085839CE3968371
:102EF00091E09783808784E0818761157105B1F047
:102F0000DB01AA5ABF4F80E090E02D913D91232B29
:102F100049F48B96880F991FDB01A80FB91FED9319
:102F2000FC93089501968031910579F70895EF9209
:102F3000FF920F931F93CF938C01C62F7A01FA0152
:102F400080819181A281B3818130F3E09F07F1E01C
:102F5000AF07B105D1F060F48115E1E09E07AE073F
:102F6000B10571F181309140A140B10571F064C0AB
:102F7000833021E0920720E1A207B105E1F183301F
:102F80009340A041B105B9F157C080913D03811133
:102F900053C020E04C2F61E1C8010E94351520E0AC
:102FA0004C2F60E1C8010E94351520E04C2F64E0F1
:102FB000C8010E94891581E080933D0381EB3DC0EB
:102FC00020E0462F61E1C8010E94351520E04C2F1A
:102FD00060E1C8010E94351510923D03F801628539
:102FE0006770C770660F660F660F6C2B82819381C6
:102FF0000E945A0C21C020E04C2F64E1C8010E94BD
:10300000351520E04C2F60E1C8010E94351564E1C0
:1030100070E080E090E00E946E0AF8016285F7019E
:1030200021812695217067704C2FF8018281938150
:103030000E94D51110923D0380E0CF911F910F9116
:10304000FF90EF900895CF92DF92EF920F931F932E
:10305000CF93DF93CDB7DEB72E970FB6F894DEBFD0
:103060000FBECDBF6C0181E090E09E878D87E12C83
:103070008E010F5F1F4F9E01235F3F4F41E0F6011E
:103080006285828193810E94FD12811151C002E00C
:1030900011E089818023D1F019861A861B861C864F
:1030A0009E01275F3F4F44E050E0612FC6010E9420
:1030B000601581110BC0AE01475F5F4F612FC601E4
:1030C0000E949717813B99F1811132C0000F1F5F59
:1030D0001830F9F611E0F6018385811740F1198661
:1030E0001A861B861C869E01275F3F4F44E050E0F6
:1030F000612FC6010E946015811117C089859A85CC
:10310000877091708130914081F48B859C858160BE
:103110009C878B87AE01475F5F4F612FC6010E947E
:103120009717813B21F0811103C01F5FD4CF80E04E
:103130002E960FB6F894DEBF0FBECDBFDF91CF91B4
:103140001F910F91EF90DF90CF9008950F931F93F1
:10315000CF93DF93FC012089211102C080E020C0C1
:10316000EC010E946C0A0C851D852E853F85DC01D3
:10317000CB01801B910BA20BB30BB7FDEFCFCE01A0
:103180000E942318182F0E946C0ADC01CB018C5975
:103190009F4FAF4FBF4F8C879D87AE87BF87812FD3
:1031A000DF91CF911F910F910895CF93DF93FC0191
:1031B000EB0180819181892B21F18281882319F192
:1031C000DA012D913C91232BE1F0A881B9819C91EA
:1031D000A381B0E0A81BB10920813181A20FB31FE8
:1031E0009C93828181508283DA018D919C91119709
:1031F00001978D939C938881998101969983888307
:10320000DCCF80E003C08381828381E0DF91CF91B6
:10321000089580914A040895CF93DF9300D01F92C0
:10322000CDB7DEB79C018091CD05843019F593E0D0
:1032300099833B832A839093E9008FEF9091E80074
:10324000815095FD06C095ED9A95F1F7000081112A
:10325000F5CF8091E80085FF0DC040E050E063E0CD
:1032600070E0CE0101960E94731D8091E8008E7778
:103270008093E8000F900F900F90DF91CF91089509
:10328000CF93DF9300D01F92CDB7DEB72091CD054D
:10329000243031F522E02983805891099B838A8369
:1032A00083E08093E9008FEF9091E800815095FDD5
:1032B00006C095ED9A95F1F700008111F5CF809148
:1032C000E80085FF0DC040E050E063E070E0CE0113
:1032D00001960E94731D8091E8008E778093E8002C
:1032E0000F900F900F90DF91CF9108952091CD0511
:1032F0002430F1F422E02093E9002FEF3091E80030
:10330000215035FD06C035ED3A95F1F70000211149
:10331000F5CF2091E80025FF0BC040E050E065E0CC
:1033200070E00E94731D8091E8008E778093E80022
:103330000895CF93DF932091CD05243049F521E006
:103340002093E90021E8215059F03091E80035FD43
:1033500007C0EFE3F1E03197F1F700C00000F3CFD1
:103360002091E80025FF14C0EC0140E050E068E047
:1033700070E00E94731D8091E8008E778093E800D2
:1033800088E0FE01A2E4B4E001900D928A95E1F795
:10339000DF91CF910895CF93C0914003C1110BC02D
:1033A0000E94D10A643C79408105910520F081E0BA
:1033B00080934003C1E08C2FCF910895FF920F932B
:1033C0001F93CF93DF93D82F0FB607FE83C0809152
:1033D000CD05843081F08091030190E00196209129
:1033E000050130E0822393232091040130E082170D
:1033F000930709F0CDC00E94CB19811110C08091B4
:10340000030190E001962091050130E0822393238F
:103410002091040130E08217930709F0B9C00E949F
:10342000C50A8C01C091E900CF709091EC00892F02
:10343000817090FD80E8C82B84E08093E90085E0EE
:10344000F82E8091EB0085FD42C08091EB0080FF5B
:103450003EC08091EE0087FF3AC0809104019091B8
:103460000301981709F457C09091E80095FF8EC0AA
:10347000E0910101F0910201E80FF11D20818F5FC1
:10348000909105018923809304012093F10080919C
:10349000E80085FDE2CF8091E80080FFDECF8091DB
:1034A000E8008E778093E800F0920001D6CF8091FB
:1034B000030190E001962091050130E082239323DF
:1034C0002091040130E08217930709F44CC0CF70BB
:1034D000C093E90040910301842F90E00196209170
:1034E000050130E0822393232091040130E082170C
:1034F000930709F450C0E0910101F0910201E40F3B
:10350000F11DD083809103018F5F90910501892384
:103510008093030140C08091E80085FF37C0D093BD
:10352000F10021E03091F3008091F20090E0932BC4
:10353000892B91F08091E80080FF0EC08091E80017
:1035400085FF03C01092F100F9CF8091E8008E77DB
:103550008093E800F0920001222309F4A8CFCF70F5
:10356000C093E90018C080910001882309F4AFCF0F
:103570000E94C50A9C018017910711F4890161CF4F
:1035800090910001915090930001F8CF20E0CACFB4
:1035900040910301B0CF80E0DF91CF911F910F9157
:1035A000FF9008958091CC05811104C00E94DF1F17
:1035B0000C943C2008951092CC050895089542E0A3
:1035C00061EC81E00E94EC1C42E061EC82E00E9430
:1035D000EC1C42E061EC83E00E94EC1C42E261ECF6
:1035E00084E00C94EC1C8091CF05833009F453C027
:1035F00030F4813071F0823009F48CC008958A3043
:1036000009F478C08B3009F45EC0893009F09AC0A3
:1036100020C08091CE05813A09F094C08091E800E5
:10362000877F8093E8008091D2059091D305892B04
:1036300021F468E082E494E003C060E080E090E080
:1036400070E00E94C01D8091E8008B778093E800B5
:1036500008958091CE05813209F074C08091D20521
:103660009091D305892B09F06DC08091E800877F88
:103670008093E8008091E80082FD05C08091CD052F
:103680008111F8CF5FC08091F10080934A0480914E
:10369000E8008B7753C08091CE05813A09F052C083
:1036A0008091D2059091D305892B09F04BC0809170
:1036B000E800877F8093E8008091E80080FFFCCFDE
:1036C0008091100136C08091CE058132D9F580916C
:1036D000D2059091D305892BA9F58091E800877FC9
:1036E0008093E8000E94211D8091D00580931001F5
:1036F0000C949A238091CE05813221F58091E800C7
:10370000877F8093E8000E94211D8091D1058093DE
:103710004B0408958091CE05813AA1F48091E80090
:10372000877F8093E8008091E80080FFFCCF809144
:103730004B048093F1008091E8008E778093E8003D
:103740000C94211D089580914A04809341031092A6
:103750004A040E9443220C949A230C94A31B0E94B7
:10376000972D8091410380934A0408950C94AF1BD8
:1037700008950C94B81B0C94B81BCF9384B7877F23
:1037800084BF0FB6F894A8958091600088618093FB
:103790006000109260000FBE90E080E80FB6F894D1
:1037A00080936100909361000FBE8EED99E10E94BD
:1037B0003E2D86E091E00E9443218CE592E00E943C
:1037C000A0020E94BB1B0E9496210E94DF1F0E9444
:1037D0003C2078940E9498218091CD05843029F076
:1037E0000E9428210E94B81BF7CF8AE492E00E9431
:1037F000A0020E94B91B88E392E00E94A002C4E0EC
:103800008091CD05853019F40E948B08F9CF0E9474
:103810009C212091E4003091E50080913E0390913D
:103820003F032817390709F468C08091E40090919C
:10383000E50090933F0380933E030E94CB198823B9
:1038400009F45BC08091CD05843009F056C08091A9
:10385000E9008F702091EC00922F917020FD90E88C
:10386000892BC093E9009091EB0090FF43C09091A9
:10387000EE0097FF3FC090910401209103012917AA
:1038800009F12091E80025FF1DC0E0910101F091B0
:103890000201E90FF11D30819F5F20910501922304
:1038A000909304013093F1009091E80095FDE3CFEF
:1038B0009091E80090FFDFCF9091E8009E77909381
:1038C000E800D9CF9091F3002091F20030E0392B3D
:1038D000232B81F09091E80090FF0CC09091E800BC
:1038E00095FF03C01092F100F9CF9091E8009E7708
:1038F0009093E8008F708093E9000E94282180CF88
:10390000292F332723303105C9F060F421303105E8
:1039100081F02230310509F041C084E790E024ECC9
:1039200032E040C021323105E1F02232310531F17F
:1039300035C082E190E028E333E034C0992781303C
:10394000910549F028F0029749F5E2E7F2E005C059
:10395000E0ECF2E002C0E0EBF2E0849190E09F0145
:1039600021C064307105D0F4660F771FFB01EA5661
:10397000FE4F2081318189E090E014C064307105F0
:1039800068F4FB01EE0FFF1FE257FE4F20813181EB
:10399000FB01E657FE4F808190E004C080E090E09C
:1039A00020E030E0FA0131832083089580E189BD71
:1039B00082E189BD09B400FEFDCF8091D8008F7DE2
:1039C0008093D8008091E00082608093E000809135
:1039D000E00081FDFCCF0895982F973068F5909313
:1039E000E900981739F07091EC002091ED005091AA
:1039F000F00003C0242F762F50E021FD02C09F5F0E
:103A0000ECCF3091EB003E7F3093EB003091ED0036
:103A10003D7F3093ED003091EB0031603093EB004F
:103A20007093EC002093ED005093F0002091EE0095
:103A300027FDE5CF80E008958F708093E90081E055
:103A400008958091CE0587FF11C08091E80082FD26
:103A500005C08091CD058111F8CF11C08091E8009B
:103A60008B770BC08091CD05882349F08091E800C9
:103A700080FFF8CF8091E8008E778093E80008956A
:103A80002091E4003091E50095E64091EC00842F10
:103A9000817040FF23C08091E80080FD1DC08091AF
:103AA000CD05882399F0853099F08091EB0085FD54
:103AB00011C04091E4005091E5002417350729F327
:103AC000915011F09A01E1CF84E0089582E00895C9
:103AD00083E0089581E0089580E008954091E80032
:103AE00042FFDDCF0895CF92DF92EF92FF920F93C6
:103AF0001F93CF93DF93EC018B017A010E94401D4D
:103B0000811135C0E114F10439F0F7018081918110
:103B1000081B190BC80FD91FC12CD12C0115110579
:103B200029F18091E80085FD18C08091E8008E772A
:103B30008093E8000E942821E114F10449F0F70184
:103B400080819181C80ED91ED182C08285E00FC0CC
:103B50000E94401D882311F30AC089918093F100CF
:103B600001501109FFEFCF1ADF0AD8CF80E0DF91B3
:103B7000CF911F910F91FF90EF90DF90CF9008951C
:103B80002091D4053091D5052617370748F06115E7
:103B9000710539F42091E8002E772093E80001C0E8
:103BA000B901FC0120E06115710579F18091CD0525
:103BB0008823F1F18530F1F18091E80083FD3CC06C
:103BC0008091E80082FD2EC08091E80080FFEBCF5D
:103BD0002091F3008091F20090E0922B6115710525
:103BE00051F08830910538F421912093F100615013
:103BF00071090196F3CF21E0089709F020E0809148
:103C0000E8008E778093E800CECF2111CFCF0AC095
:103C10008091CD05882361F0853061F08091E800C6
:103C200083FD0AC08091E80082FFF2CF80E0089512
:103C300082E0089583E0089581E008952091D405FD
:103C40003091D5052617370748F06115710539F40D
:103C50002091E8002E772093E80001C0B901FC0113
:103C600020E06115710591F18091CD05882309F45B
:103C700040C0853009F43FC08091E80083FD3DC01D
:103C80008091E80082FD2FC08091E80080FFE9CF9D
:103C90002091F3008091F20090E0922B6115710564
:103CA00059F08830910540F424912093F100319629
:103CB000615071090196F2CF21E0089709F020E0E8
:103CC0008091E8008E778093E800CBCF2111CCCF94
:103CD0000AC08091CD05882361F0853061F0809124
:103CE000E80083FD0AC08091E80082FFF2CF80E007
:103CF000089582E0089583E0089581E008951F9378
:103D0000CF93DF93CDB7DEB7AA970FB6F894DEBF97
:103D10000FBECDBFEEECF5E08091F100819325E080
:103D2000E63DF207C9F70E94F31A8091E80083FF8D
:103D30002EC18091CE059091CF05492F50E04A3099
:103D4000510508F024C1FA01EA5AFF4F0C943F32A2
:103D5000803821F0823809F01AC108C08091CA0564
:103D60009091CB05992389F082600FC08091D20594
:103D70008F70873008F00BC18093E9008091EB00D1
:103D800085FB882780F91092E9009091E800977FE1
:103D90009093E8008093F1001092F100D1C0282F99
:103DA0002D7F09F0F4C0882319F0823061F0EFC054
:103DB0008091D005813009F0EAC0933009F080E0AD
:103DC0008093CB052EC08091D00581112AC08091AF
:103DD000D2058F702FEF280F263008F0D8C08093BF
:103DE000E9002091EB0020FF1CC0933021F480916A
:103DF000EB00806214C09091EB0090619093EB0017
:103E000021E030E0A90102C0440F551F8A95E2F776
:103E10004093EA001092EA008091EB008860809362
:103E2000EB001092E9008091E800877F8093E80022
:103E30000E94211DACC08111AAC01091D0051F772E
:103E40008091E3008078812B8093E3008091E800EB
:103E5000877F8093E8000E94211D8091E80080FF09
:103E6000FCCF8091E30080688093E300111102C0D1
:103E700082E001C083E08093CD0589C08058823004
:103E800008F085C08091D0059091D1058C3D53E01C
:103E9000950779F583E08A838AE289834FB7F8949E
:103EA000DE01139620E03EE051E2E32FF0E0509374
:103EB0005700E49120FF03C0E295EF703F5FEF7081
:103EC0008E2F90E0EA3010F0C79601C0C0968D9317
:103ED0009D932F5F243149F74FBF8091E800877F82
:103EE0008093E8006AE270E0CE0101960E94C01D56
:103EF00016C06091D2057091D305AE014F5F5F4F40
:103F00000E94801CBC01892B09F441C09091E800FB
:103F1000977F9093E80089819A810E941E1E80916C
:103F2000E8008B778093E80032C0803881F580917B
:103F3000E800877F8093E8008091C9058093F100B5
:103F40008091E8008E7772CF811121C08091D005D9
:103F50009091D10599270297D4F48091E800877F4A
:103F60008093E8008091D0058093C9050E94211DAF
:103F70008091C905811106C08091E30087FD02C0D0
:103F800081E001C084E08093CD050E94DF1A80911A
:103F9000E80083FF0AC08091E800877F8093E800F3
:103FA0008091EB0080628093EB00AA960FB6F894A4
:103FB000DEBF0FBECDBFDF91CF911F9108950E944C
:103FC0004D200E945520E0EEF0E0808181608083EA
:103FD000E8EDF0E080818F77808319BCA7EDB0E039
:103FE0008C918E7F8C9380818F7E80831092CC0504
:103FF00008950F931F93CF93DF930E944D200E944B
:104000005520C8EDD0E088818F77888388818068CB
:10401000888388818F7D888319BC1092CD0510928A
:10402000C9051092CB051092CA0500EE10E0F80108
:1040300080818B7F808388818160888342E060E01B
:1040400080E00E94EC1CE1EEF0E080818E7F8083B6
:10405000E2EEF0E0808181608083808188608083EF
:10406000F80180818E7F8083888180618883DF91E1
:10407000CF911F910F910895E8EDF0E080818F7E40
:104080008083E7EDF0E080818160808384E082BFFF
:1040900081E08093CC050C94F91FE8EDF0E080817D
:1040A0008E7F80831092E20008951092DA001092C1
:1040B000E10008951F920F920FB60F9211242F93D3
:1040C0003F934F935F936F937F938F939F93AF93A0
:1040D000BF93EF93FF938091E10082FF0BC080912B
:1040E000E20082FF07C08091E1008B7F8093E100B6
:1040F0000E9427218091DA0080FF1FC08091D800A4
:1041000080FF1BC08091DA008E7F8093DA0080915F
:10411000D90080FF0DC080E189BD82E189BD09B46D
:1041200000FEFDCF81E08093CD050E94D21A05C02C
:1041300019BC1092CD050E94DB1A8091E10080FF2E
:1041400019C08091E20080FF15C08091E2008E7F4F
:104150008093E2008091E20080618093E200809190
:10416000D80080628093D80019BC85E08093CD058B
:104170000E94AD1B8091E10084FF30C08091E2007D
:1041800084FF2CC080E189BD82E189BD09B400FEB5
:10419000FDCF8091D8008F7D8093D8008091E10081
:1041A0008F7E8093E1008091E2008F7E8093E20019
:1041B0008091E20081608093E2008091C9058823AC
:1041C00011F084E007C08091E30087FD02C081E028
:1041D00001C083E08093CD050E94B61B8091E10071
:1041E00083FF24C08091E20083FF20C08091E10022
:1041F000877F8093E10082E08093CD051092C9050E
:104200008091E1008E7F8093E1008091E2008E7FBB
:104210008093E2008091E20080618093E20042E0BE
:1042200060E080E00E94EC1C0E94DE1AFF91EF919A
:10423000BF91AF919F918F917F916F915F914F91BE
:104240003F912F910F900FBE0F901F9018950895DA
:10425000CF938091CD058823A1F0C091E900CF7064
:104260009091EC00892F817090FD80E8C82B10920E
:10427000E9008091E80083FD0E947F1ECF70C0930B
:10428000E900CF91089590935104809350040895CC
:10429000E0915004F0915104309721F00190F081A9
:1042A000E02D099480E00895E0915004F0915104CC
:1042B000309721F00280F381E02D09940895E09178
:1042C0005004F0915104309721F00480F581E02DE5
:1042D0000994089520914E0430914F04281739070E
:1042E00071F090934F0480934E04E0915004F0914C
:1042F0005104309721F00680F781E02D099408954C
:1043000020914C0430914D042817390771F0909397
:104310004D0480934C04E0915004F0915104309787
:1043200021F00084F185E02D099408950C94442235
:104330000E94BC0A0C947A098F929F92AF92BF920E
:10434000CF92DF92EF92FF920F931F93CF93DF9361
:1043500000D000D01F92CDB7DEB70E94190703E549
:1043600014E0F12C8F2D0E9401084C01F801A0806F
:10437000B180A826B926A114B10439F4F3940E5FD4
:104380001F4FF0E1FF12EECF39C08091BE0581FDD5
:104390000E942E08E12CCC24C394D12CC5018C2181
:1043A0009D21892B21F1E982FA8221E0C4018C212F
:1043B0009D21892B09F420E02B830E94C50A81608E
:1043C000782F9D838C8349815A816B818D810E94D6
:1043D000472249815A816B817C818D810E94442DC5
:1043E000F801808191818C259D2591838083E394C0
:1043F000CC0CDD1CF0E1EF12D1CFC0CF8FEF898361
:104400008A831B820E94C50A8160782F9D838C83DA
:1044100049815A816B818D810E9447220E94432DE0
:104420000E941B300E944821909152048917B9F0D4
:104430000E944821809352040F900F900F900F908C
:104440000F90DF91CF911F910F91FF90EF90DF9030
:10445000CF90BF90AF909F908F900C94552D0F9060
:104460000F900F900F900F90DF91CF911F910F91B0
:10447000FF90EF90DF90CF90BF90AF909F908F9084
:1044800008950C942F080895089508950895CF93E2
:10449000DF93CDB7DEB72B970FB6F894DEBF0FBE14
:1044A000CDBF942F4F83252F588769877A878B87B5
:1044B0004A855B85452B31F02F3F31F481E09F3FEA
:1044C00019F403C081E001C080E080FD07C04F8186
:1044D000588569857A858B850E94442DDE01119669
:1044E00086E0FD0111928A95E9F785E0FE01379695
:1044F00001900D928A95E1F749815A816B817C8107
:104500008D819E810E94C2292B960FB6F894DEBF42
:104510000FBECDBFDF91CF910895CF93DF93882356
:1045200009F489C09EE7980F933018F5823829F076
:10453000833831F0C4E0D7E405C0C2E0D9E302C05B
:10454000C1E0D3E50E9448218C2309F074C08D2F6F
:104550000E94A02C0E94182D2FEF81EE94E0215094
:1045600080409040E1F700C000008D2F0E94BD2CDC
:104570000AC09CEF980F913A20F090E5980F9E3278
:1045800030F40E94A02CDF91CF910C94182D90E272
:10459000980F983050F4877091E001C0990F8A9578
:1045A000EAF7892F0E94DE2CEECF9BE5980F93301F
:1045B00080F4853A29F0863A31F083E890E005C02E
:1045C00081E890E002C082E890E0DF91CF910C9406
:1045D0006A2198E5980F973170F5883A89F0893A01
:1045E00091F08A3A99F08B3AA1F08C3AA9F08D3A81
:1045F000B1F08E3AB9F08F3AC1F080E090E017C088
:1046000082EE90E014C089EE90E011C08AEE90E056
:104610000EC085EB90E00BC086EB90E008C083EB0A
:1046200090E005C084EB90E002C087EB90E0DF9162
:10463000CF910C948021DF91CF910895CF93DF9398
:10464000882309F454C09EE7980F933008F5823808
:1046500029F0833831F0C4E0D7E405C0C2E0D9E3E3
:1046600002C0C1E0D3E50E9448218C2309F43FC079
:104670008D2F0E94A02C0E94182D2FEF81EE94E028
:10468000215080409040E1F700C000008D2F08C00D
:104690009CEF980F913A20F090E5980F9E3218F415
:1046A0000E94BD2C0DC090E2980F983068F487707E
:1046B00091E001C0990F8A95EAF7892F0E94E42CB6
:1046C000DF91CF910C94182D9BE5980F933030F427
:1046D00080E090E0DF91CF910C946A21885A873175
:1046E00030F480E090E0DF91CF910C948021DF9155
:1046F000CF910895882321F00E94DE2C0C94182D70
:104700000895882321F00E94E42C0C94182D08951C
:104710000E94FE2C0E94CD2C0E94182D0E94C030B9
:104720000E948E2F80E090E00E946A2180E090E05D
:104730000C9480210E94EE2C0C948823CF92DF925F
:10474000EF92FF920F931F93CF93DF9300D000D08F
:104750001F92CDB7DEB76C010E94572D811118C38F
:1047600085E0F601DE01119601900D928A95E1F740
:10477000F60140815181238134812115310531F0C9
:104780005F3F31F481E04F3F19F403C081E001C085
:1047900080E080FDFDC2F601F280E580E2948FE0CA
:1047A000E82249835A83FB82722F3D832C836F2D2D
:1047B0008D810E941C2C8C010E941B2C0E94152BA9
:1047C000E12FE295EF708E2F90E0FC01E05AFF4F51
:1047D0000C943F32812F807F1F70882311F0129537
:1047E000107FFF20B9F0112329F0812F0E94F12CB6
:1047F0000E94182D802F0F900F900F900F900F9008
:10480000DF91CF911F910F91FF90EF90DF90CF90AC
:104810000C948D22802F0E941E23112309F4B8C20C
:10482000812F0E94F72C0F900F900F900F900F90F8
:10483000DF91CF911F910F91FF90EF90DF90CF907C
:104840000C94182D812F807F1F70803211F01295EB
:10485000107F002319F0013009F12BC0FF20A9F0CF
:10486000EE2059F1F1E0812FEF1228C00F900F9048
:104870000F900F900F90DF91CF911F910F91FF90AC
:10488000EF90DF90CF900C94012DEE2021F021E0ED
:10489000E21609F47DC20E94042D4DC0FF20E9F00C
:1048A00085E08E1508F474C20E94DB2C812329F068
:1048B00042C0FF20F1F1E11015C0812F0F900F9041
:1048C0000F900F900F90DF91CF911F910F91FF905C
:1048D000EF90DF90CF900C947A2394E09E1508F42B
:1048E00057C229C0F601858180FF13C08F70858370
:1048F000E4CF003F09F489C108F055C180E4800F7E
:10490000803208F459C1FF2009F4EAC1EE2009F40D
:104910009AC1802F0E948D22093309F0DAC1FFEF7E
:1049200021EE84E0F15020408040E1F700C000001B
:104930002FC2E110D7C1812F59C1812F869586954D
:10494000837019F08130B9F023C2FF2019F0C8013B
:10495000937002C080E090E00F900F900F900F9046
:104960000F90DF91CF911F910F91FF90EF90DF900B
:10497000CF900C946A21FF2019F0C801937002C0F7
:1049800080E090E00F900F900F900F900F90DF91CC
:10499000CF911F910F91FF90EF90DF90CF900C94EB
:1049A0008021802FFF2019F00E94A12E02C00E94BA
:1049B000092F0F900F900F900F900F90DF91CF91D4
:1049C0001F910F91FF90EF90DF90CF900C948E2F5E
:1049D000812F837009F070C0F110DAC1202F229569
:1049E00026952770220F220F602F6F70862F90E080
:1049F000A0E0B0E06C017D01022E04C0CC0CDD1CF7
:104A0000EE1CFF1C0A94D2F704FF12C08FE090E066
:104A1000A0E0B0E004C0880F991FAA1FBB1F2A9511
:104A2000D2F7BC01CD01609570958095909503C03B
:104A300060E070E0CB011695169513701230B1F05E
:104A400040F56C297D298E299F29113031F10F9075
:104A50000F900F900F900F90DF91CF911F910F91BA
:104A6000FF90EF90DF90CF900C94302B6C297D2934
:104A70008E299F290F900F900F900F900F90DF912C
:104A8000CF911F910F91FF90EF90DF90CF900C94FA
:104A90004A2B0E94302BC701B6010F900F900F9048
:104AA0000F900F90DF91CF911F910F91FF90EF909A
:104AB000DF90CF900C94162BFF2019F0812F81707E
:104AC00001C08695882309F463C1202F229526957D
:104AD0002770220F220F602F6F70862F90E0A0E0CA
:104AE000B0E06C017D01022E04C0CC0CDD1CEE1C7C
:104AF000FF1C0A94D2F704FF12C08FE090E0A0E000
:104B0000B0E004C0880F991FAA1FBB1F2A95D2F7D7
:104B1000BC01CD01609570958095909503C060E0D3
:104B200070E0CB011695169513701230B1F040F578
:104B30006C297D298E299F29113031F10F900F901A
:104B40000F900F900F90DF91CF911F910F91FF90D9
:104B5000EF90DF90CF900C94F72B6C297D298E2954
:104B60009F290F900F900F900F900F90DF91CF9192
:104B70001F910F91FF90EF90DF90CF900C94092C34
:104B80000E94F72BC701B6010F900F900F900F9066
:104B90000F90DF91CF911F910F91FF90EF90DF90D9
:104BA000CF900C94E52B023F09F45EC008F449C095
:104BB000033F09F46CC0A7CE902F9071E92E812F8E
:104BC0008F71FF2051F00E947E2B802FEE2019F074
:104BD0008295807F73CE8F7071CE0E949F2B802F25
:104BE000EE2019F08295807F01C08F700F900F909A
:104BF0000F900F900F90DF91CF911F910F91FF9029
:104C0000EF90DF90CF900C948123FF20A9F0E4E097
:104C1000EE1508F4BDC0812F8F710F900F900F908B
:104C20000F900F90DF91CF911F910F91FF90EF9018
:104C3000DF90CF900C94C42BF5E0FE1508F4A8C0CB
:104C4000EACFFF2099F0812F8F710F900F900F9076
:104C50000F900F90DF91CF911F910F91FF90EF90E8
:104C6000DF90CF900C947E2BFF2069F3812F8F7102
:104C70000F900F900F900F900F90DF91CF911F9199
:104C80000F91FF90EF90DF90CF900C949F2BFF201F
:104C900089F0812F8F710F900F900F900F900F90D0
:104CA000DF91CF911F910F91FF90EF90DF90CF9008
:104CB0000C94692B0F900F900F900F900F90DF9135
:104CC000CF911F910F91FF90EF90DF90CF900C94B8
:104CD000642B033509F423CE073409F059C01FCEE5
:104CE000EE2021F2802F0F900F900F900F900F90D9
:104CF000DF91CF911F910F91FF90EF90DF90CF90B8
:104D00000C941E23412F4F70602FC6010E941B2E52
:104D10000F900F900F900F900F90DF91CF911F91F8
:104D20000F91FF90EF90DF90CF900C94702A0111BB
:104D30002FC0FF2069F10E949A232FEF80E792E0B5
:104D4000215080409040E1F700C000000F900F908C
:104D50000F900F900F90DF91CF911F910F91FF90C7
:104D6000EF90DF90CF900C94C42D412F4F70602FA7
:104D7000C6010F900F900F900F900F90DF91CF9181
:104D80001F910F91FF90EF90DF90CF900C941E2E0B
:104D90000F900F900F900F900F90DF91CF911F9178
:104DA0000F91FF90EF90DF90CF9008951F93CF93D6
:104DB000DF9300D000D01F92CDB7DEB7942F498388
:104DC000252F5A836B837C838D834C815D81452B9A
:104DD00031F02F3F31F481E09F3F19F403C081E0AF
:104DE00001C080E0182F117080FD31C049815A81C7
:104DF0006B817C818D810E941C2C292F22952F7024
:104E00002C3030F42A30A0F42250223030F022C06E
:104E10002C30C9F02F30B9F01DC0853A28F4843009
:104E2000C0F4823028F415C090E2980F983088F0D2
:104E3000883E30F4803E68F48450813A58F409C0CA
:104E4000803F41F406C093FB112710F903C010E026
:104E500001C011E0812F0F900F900F900F900F90D5
:104E6000DF91CF911F910895CF93DF9300D000D0B1
:104E70001F92CDB7DEB70F900F900F900F900F904D
:104E8000DF91CF910895CF93DF9300D000D000D071
:104E9000CDB7DEB726960FB6F894DEBF0FBECDBFF6
:104EA000DF91CF9108951F93CF93DF93C091730447
:104EB00016E080917404C81799F0D0E01C9FF001AF
:104EC0001D9FF00D1124EB58FB4F408151816281F1
:104ED0007381848195810E9443272196C770E9CF11
:104EE000DF91CF911F9108954091A5045091A604A0
:104EF0006091A7047091A8048091A9049091AA04DC
:104F00000C9443270F931F93CF93DF938091AA04B0
:104F100082958F7009F05DC08091A704882309F401
:104F200058C080917304109174046091A50470912D
:104F3000A604C091A804D091A90491E06F3F09F0A4
:104F400090E0292F06E0811709F443C0209721F053
:104F50007F3F21F030E003C031E001C0322F90E00C
:104F600030FD34C0089FF001099FF00D1124DF01CE
:104F7000AB58BB4F11963C911197371327C03C910A
:104F8000361324C012963C91129731111FC013960C
:104F90004D915C9114974C1B5D0B483C5105B0F44E
:104FA0008091AA048F7080618093AA04E658FB4F19
:104FB00080818F708061808385EA94E00E949E23C7
:104FC000DF91CF911F910F910C9453270196877019
:104FD000BACFDF91CF911F910F9108959F92AF9219
:104FE000BF92CF92DF92EF92FF920F931F93CF93D6
:104FF000DF93CDB7DEB761970FB6F894DEBF0FBE73
:10500000CDBF8C0185E0F801DE011D9601900D9267
:105010008A95E1F7F80140815181F280C380D48004
:105020009091A5046091A6042091A8043091A90450
:105030002115310531F06F3F31F481E09F3F19F4C4
:1050400003C081E001C080E0F82FF1709F2E80FD49
:1050500052C185EAA82E84E0B82EE090A704F6019C
:10506000E21BF30BEE2009F4E8C08091AA04E83CAF
:10507000F10508F0A4C0282F207F09F053C0561373
:1050800013C0491311C0EF2CF1100EC08F70806156
:105090008093AA040E947427C5010E949E238091D8
:1050A000AA04F80185835BC1C114D10431F05F3FCC
:1050B00031F481E04F3F19F403C081E001C080E08A
:1050C00080FD03C081E08F2502C080E090E0F82FD2
:1050D000F170EF2E80FF1CC0809173042091740446
:1050E00036E0821709F418C190E0389FF001399F2B
:1050F000F00D1124EB58FB4F6181561306C06081FF
:10510000461303C06281F61203C001968770E9CF8F
:10511000EF2CFF2009F423C18091AA0481608093C1
:10512000AA0462C0561306C0491304C0F11002C09D
:10513000F801A7C04D875E87FF867C2DD98AC88A73
:105140006F2D89890E94D626882399F1FF2089F145
:105150002091AA04822F82958F7090E0029774F0BC
:105160008091A5049091A60498878F831986DB8689
:10517000CA862C87CE0107960E949E2386E0F801FE
:10518000A5EAB4E001900D928A95E1F70E9482278A
:105190000E94742711C0561749F14D875E87FF861C
:1051A0007C2DD98AC88A6F2D89890E94D6268111C3
:1051B0002CC0C8010E949E23EE24E394D0C0282F67
:1051C000207F49F77C2DD98AC88A6F2D89890E9452
:1051D000342785EA94E00E949E2386E0F50111922F
:1051E0008A95E9F70E947427E12CB9C04913D5CFFD
:1051F000F110D3CFF8018583C8010E949E2386E079
:10520000F50111928A95E9F7AAC0FF2091F2209149
:10521000AA04822F82958F7090E002970CF4AECF93
:105220008091A5049091A6049A8389831B82DD82D4
:10523000CC822E83CE0101969FCFE83CF10508F089
:105240004BC0EF2CFF2009F4B4CF561330C04913E4
:105250002EC02091AA0420FD21C0822F82958F703C
:10526000482F50E041155105C9F0F80125834F3012
:10527000510541F08F5F982F9295907F822F8F700C
:10528000892B8583C8010E949E2386E0F801A5EA48
:10529000B4E001900D928A95E1F72AC086E0F8010A
:1052A000A5EAB4E001900D928A95E1F758C04D87C8
:1052B0005E87FF867C2DD98AC88A6F2D89890E94D6
:1052C000D62681115BCF8091AA0481608093AA04C5
:1052D000C8010E949E2343C07C2DD98AC88A6F2DA5
:1052E00089890E94342786E0F50111928A95E9F7B1
:1052F0000E94742734C0FF2009F45BCF4D875E877E
:10530000FF867C2DD98AC88A6F2D89890E94D6266E
:10531000882309F44ECF32CF7C2DD98AC88A6F2DCD
:1053200089890E941C2C292F22952F70223028F465
:105330009F7039F0811105C00BC0243028F49F7094
:1053400049F4805E883020F0C8010E949E239E2C84
:10535000E92C05C0F8019581907F99F7F9CF8E2D42
:1053600061960FB6F894DEBF0FBECDBFDF91CF912F
:105370001F910F91FF90EF90DF90CF90BF90AF9073
:105380009F9008951F93CF93DF93CDB7DEB72C97EF
:105390000FB6F894DEBF0FBECDBF4F835887698725
:1053A0007A878B879C87CE0107960E94EE278823F9
:1053B000D1F09F8188852A853B85232B31F08F3F53
:1053C00031F481E09F3F19F403C081E001C080E027
:1053D00080FD47C04F81588569857A858B859C857E
:1053E0000E9443273EC086E0FE013796DE011196FB
:1053F00001900D928A95E1F7FF81E8856A857B85AA
:105400006115710531F0EF3F31F481E0FF3F19F490
:1054100003C081E001C080E080FD23C020917404BE
:1054200030E0C9010196877099274091730450E0DC
:1054300084179507F1F1F983EA837D836C8396E005
:10544000929FD001939FB00D1124AB58BB4FFE012A
:10545000319601900D929A95E1F7809374040E9421
:10546000532716E08091730490917404891771F1A9
:10547000189FC00111248B589B4F0E94EE27882350
:1054800029F1E09173041E9FF0011124EB58FB4FAA
:105490004081518162817381848195810E9443277B
:1054A0008091730490E0019687709927809373042C
:1054B000D9CF0E949A231092740410927304E5EAE3
:1054C000F4E086E0DF011D928A95E9F72C960FB68D
:1054D000F894DEBF0FBECDBFDF91CF911F9108952D
:1054E000DF92EF92FF920F931F93CF93DF93FC0114
:1054F000892B09F488C0E12CF12CDD24D394EF0131
:1055000021968491853709F460C058F4843708F0F7
:105510004EC0843008F068C08130D1F0823071F123
:1055200072C0883709F45BC050F4863709F453C061
:10553000873709F068C08E2D0E94EB2C52C09CE783
:10554000980F903708F05FC08F770E941E234EC0DF
:105550008F010E5F1F4FFE01849190E2980F9830EB
:1055600050F48770FD2D01C0FF0F8A95EAF78F2F49
:105570000E94F12C15C00E948D2214C08F010E5F75
:105580001F4FFE01849190E2980F983068F4877065
:10559000FD2D01C0FF0F8A95EAF78F2F0E94F72C8F
:1055A0000E94182DE80122C00E941E23FBCFCF01CC
:1055B0000296FE01C491CC2361F0EFE9FFE0319740
:1055C000F1F700C00000C150F6CFCF010296FE01F6
:1055D000F490EC010BC00E94DB2CE82E07C00E9467
:1055E000EE2C0E94182D02C00E948D228F2D882340
:1055F00041F0EFE9FFE03197F1F700C00000815082
:10560000F6CFFE017CCFDF91CF911F910F91FF90DC
:10561000EF90DF9008956093AB057093AC05809395
:10562000AD059093AE050C94542D08950F931F93E0
:105630000091AF051091B0052091B1053091B205F0
:10564000602B712B822B932B6093AF057093B00569
:105650008093B1059093B2051F910F910C94532D37
:105660000F931F930091AF051091B0052091B105E4
:105670003091B20560237123822393236093AF0599
:105680007093B0058093B1059093B2051F910F916F
:105690000C94532D0F931F930091AF051091B005FB
:1056A0002091B1053091B205602771278227932799
:1056B0006093AF057093B0058093B1059093B205E8
:1056C0001F910F910C94532D60E070E0CB010C946E
:1056D0000B2B0F931F9341E050E060E070E08A01D4
:1056E0009B0104C0000F111F221F331F8A95D2F7A0
:1056F000C901B8011F910F910C940B2B0F931F93AD
:1057000041E050E060E070E004C0440F551F661FA8
:10571000771F8A95D2F78091AB059091AC05A09147
:10572000AD05B091AE058A019B01082B192B2A2BE0
:105730003B2BC901B8011F910F910C940B2B0F93B8
:105740001F9341E050E060E070E004C0440F551F3B
:10575000661F771F8A95D2F7409550956095709592
:105760008091AB059091AC05A091AD05B091AE05CF
:105770008A019B01082319232A233B23C901B8016D
:105780001F910F910C940B2B0F931F9341E050E04E
:1057900060E070E004C0440F551F661F771F8A95B4
:1057A000D2F78091AB059091AC05A091AD05B09179
:1057B000AE058A019B01082719272A273B27C90123
:1057C000B8011F910F910C940B2B0F931F93009115
:1057D000AB051091AC052091AD053091AE05602B65
:1057E000712B822B932B1F910F910C940B2B0F93EA
:1057F0001F930091AB051091AC052091AD05309140
:10580000AE0560237123822393231F910F910C9483
:105810000B2B0F931F930091AB051091AC052091BA
:10582000AD053091AE0560277127822793271F9120
:105830000F910C940B2B08958F929F92AF92BF9271
:10584000DF92EF92FF920F931F93CF93DF9300D0DD
:1058500000D01F92CDB7DEB76B837C838D838A0126
:105860008C819D81892B31F01F3F31F481E04F3FC6
:1058700019F403C081E001C080E080FF03C080E034
:1058800090E04DC08B818823D1F18090AB05909042
:10589000AC05A090AD05B090AE058091AF0590919C
:1058A000B005A091B105B091B205882A992AAA2A1B
:1058B000BB2A8FE1E82EF12CD501C4010E2C04C0C7
:1058C000B695A795979587950A94D2F780FD06C05F
:1058D00081E0E81AF10880F7D12C07C0DE2CB8016E
:1058E0008E2D0E94F32D019799F380E1189FF0010E
:1058F0001124E555FB4FE00FF11DD08209C080E176
:10590000189FF0011124E555FB4FE00FF11DD080E9
:1059100009831A8369817A818D2D0E94F32D0F905E
:105920000F900F900F900F90DF91CF911F910F91DB
:10593000FF90EF90DF90BF90AF909F908F90089571
:105940002091110130911201F90132969FEF40E050
:105950005191851789F09F3F19F4511101C0942F7F
:105960004F5F4630A9F79F3F39F0F901E90FF11D6C
:1059700097FDFA95828308950895E0911101F091C1
:1059800012019F012A5F3F4F9281891301C0128249
:105990003196E217F307C1F7089581E090E0E091B6
:1059A0001101F0911201E80FF91F10820196883061
:1059B0009105A9F708958091BD0508959091BD05C1
:1059C000892B8093BD05089580959091BD0589230D
:1059D0008093BD0508958093BD0508951092BD057F
:1059E00008959091BC05892B8093BC0508958095FE
:1059F0009091BC0589238093BC0508951092BC0545
:105A000008958093B30508951092B3050895809189
:105A1000110190911201FC0131969C01285F3F4FCA
:105A200080E0919191118F5FE217F307D1F708950C
:105A3000E0911101F09112018091BD058083E09108
:105A40001101F091120190818091BC05892B808316
:105A50008091B305882361F0E0911101F09112016A
:105A60009081892B80830E94072D81111092B305AC
:105A700080911101909112010C94542190939F01F7
:105A800080939E0108950895CF93DF9300D000D0B6
:105A90001F92CDB7DEB70F900F900F900F900F9021
:105AA000DF91CF910895089508950C94412280E0EC
:105AB00008958091CD05843021F11092BF0520E436
:105AC00088E190E00FB6F894A895809360000FBE2F
:105AD0002093600083B7817F846083BF83B7816038
:105AE00083BF7894889583B78E7F83BF0FB6F89471
:105AF000A89580916000886180936000109260009A
:105B00000FBE0895CF930E9445220E9419070E945C
:105B10004622C0E08C2F0E940108892B29F4CF5F18
:105B2000C031C1F780E001C081E0CF9108950E94AB
:105B300043220C949A231F920F920FB60F921124B6
:105B40008F939F93AF93BF938091BF05811113C033
:105B50008091340390913503A0913603B0913703BF
:105B60004196A11DB11D8093340390933503A093FA
:105B70003603B0933703BF91AF919F918F910F90F0
:105B80000FBE0F901F9018950E94DF1FF89487E7B3
:105B900097E7909301088093000887E090EBDC0181
:105BA0008093D6059093D705A093D805B093D905D7
:105BB0009CE088E10FB6F894A895809360000FBE32
:105BC00090936000FFCFE82FF0E080E1989FE00D18
:105BD000F11D1124E052FF4F8491982F92959F70F0
:105BE0008F7097700895CF93C82FCB010E94E32D3B
:105BF00040E1949F90011124282B203831051CF09E
:105C000080E090E016C09770E92FF0E098E0C99F1F
:105C1000E00DF11D112494E0EE0FFF1F9A95E1F7BE
:105C20008F70E80FF11DEE0FFF1FE050F8498591CE
:105C30009491CF91089580E090E008950895809127
:105C4000C20580FF0BC06091160185E0689FB0011E
:105C5000112475956795759567952BC081FF09C0CF
:105C60006091160185E0689FB001112475956795D4
:105C700020C082FF07C06091160185E0689FB001D7
:105C8000112417C09091C3059923D1F0609115019B
:105C9000961788F72091160185E0289F900111241E
:105CA000929FA001939F500D112470E0CA010E94A1
:105CB0002B326038710540F46115710519F406C086
:105CC00065E070E0862F08958FE7089581E00895DC
:105CD0008091C20580FF08C06091140170E0759545
:105CE00067957595679521C081FF06C06091140185
:105CF00070E07595679519C082FF04C0609114012A
:105D000070E010C09091C305992399F06091130140
:105D10009617A0F780911401899FC001112470E0AB
:105D20000E942B326038710540F46115710519F439
:105D300006C061E070E0862F08958FE7089581E046
:105D40000895803F21F40E941F2E819504C0813F59
:105D500029F40E941F2E8093C6050895823F21F4E6
:105D60000E941F2E819504C0833F29F40E941F2E9C
:105D70008093C5050895893F19F40E94682E05C0D7
:105D80008A3F31F40E94682E81958093C70508955B
:105D90008B3F21F40E94682E819504C08C3F29F42A
:105DA0000E94682E8093C8050895843F21F4809155
:105DB000C405816017C0853F21F48091C4058260CD
:105DC00011C0863F21F48091C40584600BC0873FD9
:105DD00021F48091C405886005C0883F31F480912A
:105DE000C40580618093C40508958D3F21F480919E
:105DF000C20581600BC08E3F21F48091C205826094
:105E000005C08F3F29F48091C20584608093C2054C
:105E10000895803F39F48091C60587FF6CC01092C9
:105E2000C60569C0813F29F48091C6051816BCF3E8
:105E300062C09091C505823F29F497FF5CC0109223
:105E4000C50559C0833F19F41916CCF354C0893FD6
:105E500041F48091C70518160CF04DC01092C7058B
:105E60004AC08A3F29F48091C70587FF44C0F6CF16
:105E70008B3F39F48091C80587FF3DC01092C8055B
:105E80003AC08C3F29F48091C8051816BCF333C082
:105E9000843F21F48091C4058E7F17C0853F21F493
:105EA0008091C4058D7F11C0863F21F48091C40587
:105EB0008B7F0BC0873F21F48091C405877F05C08D
:105EC000883F31F48091C4058F7E8093C40513C050
:105ED0008D3F21F48091C2058E7F0BC08E3F21F44F
:105EE0008091C2058D7F05C08F3F29F48091C20546
:105EF0008B7F8093C2058091C50581110EC0809172
:105F0000C60581110AC08091C705811106C0809124
:105F1000C805811102C01092C30508958091BE0585
:105F200083FF7EC086E594E00E94A0028091C405B4
:105F30001F928F9381E594E09F938F930E94390382
:105F40008FE494E00E94A0028091C505282F082EBE
:105F5000000C330B3F938F938CE494E09F938F93CB
:105F60000E9439038AE494E00E94A0028091C60551
:105F7000282F082E000C330B3F938F9387E494E077
:105F80009F938F930E94390385E494E00E94A002BE
:105F90008091C705282F082E000C330B3F938F9359
:105FA00082E494E09F938F930E94390380E494E00D
:105FB0000E94A0028091C805282F082E000C330BE8
:105FC0003F938F938DE394E09F938F930E943903C7
:105FD0008AE394E00E94A0028091C3051F928F93F0
:105FE00087E394E09F938F930E94390385E394E0C5
:105FF0000E94A0028091C2051F928F9382E394E0D9
:106000009F938F930E9439038FE294E00E94A00235
:106010008DB79EB74C960FB6F8949EBF0FBE8DBF3E
:1060200084EC95E00E945F210E94C50A9093C1050F
:106030008093C00508951F93CF93DF938091C0058F
:106040009091C1050E94DD0AAC019091C30599238E
:1060500021F02091170130E006C0209118018AE05C
:10606000289F900111244217530708F485C080919E
:10607000C505C091C605D091C7051091C80581110D
:1060800007C0C11175C0D11173C0111171C074C0A6
:106090009F3F19F09F5F9093C305181624F40E9448
:1060A0001F2E8093C5058091C50587FF05C00E94FE
:1060B0001F2E81958093C5051C1624F40E941F2E67
:1060C0008093C6058091C60587FF05C00E941F2EDC
:1060D00081958093C6056091C505662331F1C09115
:1060E000C605CC2311F1062E000C770B880B990BFB
:1060F0000E94093123E333E343E35FE30E94BE31AF
:106100000E94D1306093C5056C2FCC0F770B880BA4
:10611000990B0E94093123E333E343E35FE30E94D9
:10612000BE310E94D1306093C6051D1624F40E9432
:10613000682E8093C7058091C70587FF05C00E9420
:10614000682E81958093C705111624F40E94682E4D
:106150008093C8058091C80587FF05C00E94682EFE
:1061600081958093C805DF91CF911F910C948E2F5C
:106170009F3F09F08FCFA0CFDF91CF911F9108955E
:10618000E4ECF5E085E0DF011D928A95E9F71092D5
:10619000C3051092C20508950E94443108F481E0BD
:1061A00008950E94D8306894B1110C94B3310895C9
:1061B0000E94983188F09F5798F0B92F9927B751CE
:1061C000B0F0E1F0660F771F881F991F1AF0BA959B
:1061D000C9F714C0B13091F00E94B231B1E0089516
:1061E0000C94B231672F782F8827B85F39F0B93F08
:1061F000CCF3869577956795B395D9F73EF490954E
:106200008095709561957F4F8F4F9F4F0895E894CB
:1062100009C097FB3EF490958095709561957F4FEE
:106220008F4F9F4F9923A9F0F92F96E9BB2793959C
:10623000F695879577956795B795F111F8CFFAF4AC
:10624000BB0F11F460FF1BC06F5F7F4F8F4F9F4FDD
:1062500016C0882311F096E911C0772321F09EE83B
:10626000872F762F05C0662371F096E8862F70E0A1
:1062700060E02AF09A95660F771F881FDAF7880F7B
:106280009695879597F90895990F0008550FAA0BD1
:10629000E0E8FEEF16161706E807F907C0F0121639
:1062A0001306E407F50798F0621B730B840B950B3C
:1062B00039F40A2661F0232B242B252B21F4089591
:1062C0000A2609F4A140A6958FEF811D811D08952E
:1062D00097F99F6780E870E060E008959FEF80EC99
:1062E000089500240A94161617061806090608953C
:1062F00000240A9412161306140605060895092EA2
:106300000394000C11F4882352F0BB0F40F4BF2B10
:1063100011F460FF04C06F5F7F4F8F4F9F4F089550
:1063200057FD9058440F551F59F05F3F71F0479546
:10633000880F97FB991F61F09F3F79F0879508952B
:10634000121613061406551FF2CF4695F1DF08C04A
:10635000161617061806991FF1CF86957105610567
:1063600008940895E894BB2766277727CB0197F90F
:1063700008950E94443108F48FEF08950E94D131AE
:106380000C947F310E94713138F00E94783120F0F6
:10639000952311F00C9468310C946E3111240C94F7
:1063A000B3310E94903170F3959FC1F3950F50E087
:1063B000551F629FF001729FBB27F00DB11D639FB7
:1063C000AA27F00DB11DAA1F649F6627B00DA11D5D
:1063D000661F829F2227B00DA11D621F739FB00D03
:1063E000A11D621F839FA00D611D221F749F332773
:1063F000A00D611D231F849F600D211D822F762F0C
:106400006A2F11249F5750409AF0F1F088234AF0E8
:10641000EE0FFF1FBB1F661F771F881F9150504054
:10642000A9F79E3F510580F00C9468310C94B3316C
:106430005F3FE4F3983ED4F3869577956795B795DB
:10644000F795E7959F5FC1F7FE2B880F911D9695F5
:10645000879597F9089597FB072E16F4009407D0B7
:1064600077FD09D00E94453207FC05D03EF4909597
:1064700081959F4F0895709561957F4F0895EE0F18
:10648000FF1F0590F491E02D0994AA1BBB1B51E15D
:1064900007C0AA1FBB1FA617B70710F0A61BB70B94
:1064A000881F991F5A95A9F780959095BC01CD0139
:0664B0000895F894FFCFEF
:1064B6000542030000FF09199919761940190C19AC
:1064C60001B4052808140A321E66756C6C006C6FE0
:1064D600770000000000D60500000000050400005B
:1064E60000007704420392030604AD034403450308
:1064F600B003B503BA0386038F03C203FEFF000091
:10650600FB0300000000DA09000000004A0A500AF6
:10651600460A490A400A430A430A000000006B0B78
:10652600120BCB0B00000000B41542031315A6187E
:106536000B15021745030E154703404D3622EF0390
:0E654600A2036C034A03D602EF0208032103EE
:106800008800EA44E944E244040005000600070069
:10681000080009000A000B000C000D000E000F001C
:1068200010001100120013001400150016001700CC
:10683000180019001A001B001C001D001E001F007C
:10684000200021002200230024002500260027002C
:10685000280029002A002B002C002D002E002F00DC
:10686000300031003200330034003500360037008C
:10687000380039003A003B003C003D003E003F003C
:1068800040004100420043004400450046004700EC
:10689000480049004A004B004C004D004E004F009C
:1068A000500051005200530054005500560057004C
:1068B000580059005A005B005C005D005E005F00FC
:1068C00060006100620063006400F1A18500670060
:1068D000680069006A006B006C006D006E006F005C
:1068E0007000710072007300890087008A008B00BD
:1068F000E000E100E200E300E400E500E600E7007C
:106900000100010001000100EA4401000100E2442D
:106910000100010001000100460001004A004B0097
:10692000010001004700480001000100E9440100A6
:106930000100010001000100010001003A003B00DC
:106940003C003D003E003F0040004100420043004B
:10695000010035004C0001000100440045005200D8
:1069600049000100010050004F0029004D004E0079
:1069700051000100010001000100010001000100BF
:1069800001000100010001000100010001000100FF
:1069900000E00100010001000100010001004D00C4
:1069A0004A004E004B0001000100010001000100FF
:1069B00001000100010001000100010001000100CF
:1069C00001000100010001000100010001000100BF
:1069D00001000100010001000100010001000100AF
:1069E0000100010001000100490001000100010057
:1069F000010001000100010001000100010001008F
:00000001FF
